:020000040800F2
:1000000000040020E1010008E3010008E30100080A
:10001000E3010008E3010008E3010008E301000830
:10002000E3010008E3010008E3010008B12600082D
:10003000E3010008E3010008E3010008E301000810
:10004000E3010008E3010008E3010008E301000800
:10005000E3010008E3010008013800082D3800081A
:100060005938000885380008B1380008E301000855
:10007000E3010008E3010008E3010008E3010008D0
:10008000E3010008E3010008E3010008E3010008C0
:10009000E3010008E3010008E3010008DD3800087F
:1000A000E3010008E3010008E3010008E3010008A0
:1000B0001D360008E3010008E3010008E301000821
:1000C000E3010008E3010008E3010008E301000880
:1000D000E30100081D10000831100008E3010008CA
:1000E00045390008E3010008E3010008E3010008C6
:1000F000E3010008E3010008E3010008E301000850
:10010000E3010008E3010008E3010008E30100083F
:10011000E301000845100008E3010008E3010008BE
:10012000E3010008E3010008E3010008E30100081F
:10013000E3010008E3010008E3010008E30100080F
:10014000E3010008E3010008E30100089D2D000819
:10015000E3010008E3010008E3010008E3010008EF
:10016000E3010008E3010008E3010008E3010008DF
:10017000E3010008E3010008E3010008E3010008CF
:10018000E3010008E3010008E3010008E3010008BF
:10019000E3010008E3010008E3010008E3010008AF
:1001A000E3010008E3010008E3010008E30100089F
:1001B000E3010008E3010008E3010008E30100088F
:1001C000E3010008E3010008E3010008E30100087F
:1001D000E3010008E3010008E3010008E30100086F
:1001E00002E000F000F8FEE772B6394880F30888B4
:1001F000384880F3098838484EF60851CEF200019D
:10020000086040F20000CCF200004EF63471CEF2ED
:1002100000010860BFF34F8FBFF36F8F40F2000003
:10022000C0F2F0004EF68851CEF200010860BFF334
:100230004F8FBFF36F8F4FF00000E1EE100A4EF6C4
:100240003C71CEF200010860062080F31488BFF3F1
:100250006F8F02F06BFA03F077F94FF055301F49BA
:100260001B4A91423CBF41F8040BFAE71C49194A6A
:1002700091423CBF41F8040BFAE71A491A4A1B4B5A
:100280009A423EBF51F8040B42F8040BF8E70020F5
:100290001749184A91423CBF41F8040BFAE702F0B3
:1002A00049FA03F0ADF9144C144DAC4203DA54F89A
:1002B000041B8847F9E700F03FF8114C114DAC42A0
:1002C00003DA54F8041B8847F9E702F031BA00005A
:1002D000000400200024002000000008000000208E
:1002E00000040020C03D0008002400202824002035
:1002F0002824002088410020E0010008E0010008D7
:10030000E0010008E00100082DE9F04F2DED108A12
:10031000C1F80CD0C3689D46BDEC108ABDE8F08FD3
:10032000002383F311882846A047002001F068FECF
:1003300001F018FE00DFFEE71A4B6FF0780270B58F
:1003400000241A700F225C709C70DC701C715C7150
:100350009C71DC711C725C729A72DC7202F07EF924
:10036000064602F09FF9054650B90F4B9E4217D042
:1003700001339E4241F2883412BF05460024012514
:10038000002002F071F90DB100F0B4F800F044FD66
:1003900000F026FC204600F00BF900F0ABF8F9E77E
:1003A0000446EDE728240020010007B008B500F05E
:1003B00095FBA0F120035842584108BD07B5054BF5
:1003C00002211B88ADF8043001A800F0F3FB03B054
:1003D0005DF804FB443A0008064991F8243033B133
:1003E00000230822086A81F8243000F01BBC012099
:1003F000704700BF482400202DE9F84F234C94F8A3
:1004000024300546884617468BBB2E46DFF87C9085
:10041000002F38D094F824A0BAF1000F05D1202283
:10042000FF214846266200F0E5FCCAF10805BD42FE
:1004300028BF3D465FFA85FBAD0041462A4604EBE6
:100440008A0000F0ADFC94F82430A7EB0B079B4426
:100450005FFA8BFBBBF1080F2E44A844FFB284F86F
:1004600024B0D5D1FFF7B8FF0028D1D108E0266A23
:1004700006EB8306B042C9D0FFF7AEFF0028C4D117
:100480000020BDE8F88F0120BDE8F88F4824002047
:1004900010B5202383F311881248C3680BB101F013
:1004A00035FE0023104A0F484FF47A7101F0F2FD37
:1004B000002383F311880D4C236813B12368013B9B
:1004C0002360636813B16368013B6360084B1B786A
:1004D00033B9636823B9022000F058FC322363600B
:1004E00010BD00BF342400209104000878290020AA
:1004F0007024002010B5254B254953F8042F0132F4
:1005000000D110BD8B42F8D1224C234B22689A4275
:100510003AD9224B9B6803F1006303F580339A427A
:1005200032D2002000F076FB1D4B0220187000F044
:1005300023FC1C4B1A6C00221A64196E1A66196E81
:10054000596C5A64596E5A665A6E5A6942F0800262
:100550005A615A6922F080025A615A691A6942F056
:1005600000521A611A6922F000521A611B6972B6B0
:100570000D4A0E4B13601B682268202181F31188FD
:100580009D4683F30888104710BD00BFFCFF00089C
:100590001C00010804000108FFFF000828240020B7
:1005A000702400200038024008ED00E0000001083F
:1005B0002DE9F04FB04C97B020228146FF210EA8C4
:1005C000A66800F017FCAD4A1378A346A3B9AC485F
:1005D0000121C3601170202383F31188C3680BB11C
:1005E00001F094FD0023A74AA5484FF47A7101F069
:1005F00051FD002383F31188B9F1000F02D0A24B03
:10060000C3F80090A14BA04A00241C7054602546FA
:1006100027469846012000F0AFFBB9F1000F00F02B
:100620002282994B1B68002B40F01D8217B0BDE859
:10063000F08F0220FFF7BAFE002840F00E82944BA4
:100640001B88ADF82430022109A800F0B3FAE1E7D5
:100650004FF47A7000F042FA031E0193EFDB0220A0
:10066000FFF7A4FE82460028E9D0019B581E04280B
:1006700000F2F581DFE800F0030D1013160016A854
:10068000052340F8343D042100F094FA5446002735
:1006900052E004217848F7E704217E48F4E704217A
:1006A0007D48F1E71C24204600F0B6FA0434099096
:1006B000042109A800F07EFA2C2CF4D1E6E7002DE5
:1006C000BDD0002CBBD00220FFF770FE05460028ED
:1006D00000F0C781012000F09DFA022088F8000098
:1006E00000F04AFB0024E3B21846019300F0A2FA9E
:1006F000824648B1019B184600F0ACFA013400284C
:10070000F1D12C46654B9BE70123022088F800308D
:1007100000F028FB5646DBF808309E4206D23046F1
:1007200000F07AFA0130ECD10436F4E7564B00269B
:1007300088F800605E602C4600F064FB1DB1002C60
:1007400018BF4FF00009FFF739FE63E7002D3FF4B3
:1007500076AF002C3FF473AF022088F8000000F061
:100760000BFB322000F0BAF9B0F1000AC0F2798137
:100770001AF0030540F07581DBF8082006EB0A0348
:10078000934200F26E81BAF5807F00F26A81444B99
:10079000019355450DDA4FF47A7000F09FF90290FD
:1007A000029A002AC0F25D81019B029AEA54013547
:1007B000EEE7C820FFF7FAFD0546002800F051815A
:1007C0001F2E11D8C6F12004544528BF54460EAB45
:1007D00026F0030022463249184400F0E1FA22468E
:1007E000FF212F4800F006FB4FEAAA0A5FFA8AF2BF
:1007F0002B493046FFF700FE0446002881D006EB67
:100800008A06054698E70220FFF7D0FD00283FF44E
:1008100016AFFFF7E1FD00283FF411AF002292462A
:10082000DBF808309A4259D21F2A1ED80E9B01339A
:100830001BD022F0030316A90B4453F8203C099364
:100840001848436883B3174800210DF1240E11F8AE
:100850000E3083EA0A03DBB2013150F82330042959
:1008600083EA1A2AF3D10432DAE71046019200F043
:10087000D3F9019A0990E3E7282400207425002089
:1008800034240020910400087829002070240020DE
:10089000463A00082C24002030240020483A000862
:1008A000742400207825002019464FF0080E11F01E
:1008B000010F4FEA51011FBF81F06D4181F43801F2
:1008C00081F4034181F02001BEF1010EEFD140F827
:1008D00023100133B3F5807FE6D1B4E716A80421D5
:1008E00040F84CAD00F066F926E716A8002340F862
:1008F000343D642100F02AF900287FF4A0AE0220E4
:10090000FFF754FD00283FF49AAE099800F0B4F9BF
:1009100016AB43F8480D04211846E3E716A8002358
:1009200040F8343D642100F011F900287FF487AECF
:100930000220FFF73BFD00283FF481AE099800F04C
:10094000A9F916AB43F8440DE5E70220FFF72EFDA9
:1009500000283FF474AE00F0A3F916AB43F8400D45
:10096000D9E70220FFF722FD00283FF468AE09A96D
:10097000142000F09BF9824616A8042140F83CADF3
:1009800000F018F9514609A8ACE7322000F0A6F8AB
:10099000B0F1000AFFF653AE1AF0030F7FF44FAE2A
:1009A000DBF808200AEB070393423FF648AE02202B
:1009B000FFF7FCFC00283FF442AE2AF0030ABA44D9
:1009C000BA453FF4B9AE384600F026F90421089044
:1009D00008A800F0EFF80437F2E74FF47A70FFF759
:1009E000E5FC00283FF42BAEFFF7F6FC00283FF4AF
:1009F00089AE0E9B01330CD008220EA90020FFF710
:100A0000FBFC00283FF47EAE2022FF210EA800F060
:100A1000F1F9FFF7D3FC304801F0F8FA06E616A822
:100A2000002340F8343D642100F090F8824600280D
:100A30007FF405AE0220FFF7B9FC00283FF4FFADBC
:100A4000FFF7BCFC41F2883001F0E0FA099800F0B1
:100A500021FAD14600F0D6F9DCE505466CE6002720
:100A6000EDE52546EBE5002000F038F80290029B0A
:100A7000002BFFF6D2AD012000F074F9029B213B60
:100A8000122B3FF6C7AD01A252F823F0330600083F
:100A900051060008BF0600081506000815060008E4
:100AA000150600084D0700088B0900080708000814
:100AB000EB0800081D0900084B090008150600088E
:100AC0006309000815060008DB090008390700085B
:100AD000150600081F0A0008A08601002DE9F3474B
:100AE00002AE00244FF47A7506F8014D144FDFF87A
:100AF0005880454397F900305A1C5FFA84F901D0B9
:100B0000A34212D158F8240003680122D3F820A090
:100B100031462B46D047012807D10A4B9DF80700E4
:100B200083F8009002B0BDE8F0870134042CE1D1D5
:100B30004FF4FA7001F06AFA4FF0FF30F2E700BFAD
:100B40000024002098290020883A00082DE9F04769
:100B50004FF47A75144FDFF8588006464D43002451
:100B600097F900305A1C5FFA84F901D0A34210D1E2
:100B700058F8240003680422D3F820A031462B46FD
:100B8000D047042805D1094B83F800900020BDE828
:100B9000F0870134042CE3D14FF4FA7001F036FAF7
:100BA0004FF0FF30BDE8F087002400209829002096
:100BB000883A000830B4074B1A78074B53F82240A4
:100BC0002368DD69054B0A46AC460146204630BC29
:100BD000604700BF98290020883A0008A0860100DD
:100BE00070B501F05BFC094C094E2070002530689F
:100BF0002378834208D901F04BFC33680544013364
:100C0000B5F5803F3360F2D370BD00BF9929002055
:100C10008029002001F0ECBC00F1006000F580307C
:100C20000068704700F10060920000F5803001F02C
:100C300077BC0000054B1A68054B1B789B1A834252
:100C400002D9104401F024BC002070478029002004
:100C50009929002038B5074D04462868204401F042
:100C60001FFC28B928682044BDE8384001F030BC9A
:100C700038BD00BF8029002010F0030308D1B0F573
:100C8000007F05D800F10050A0F5084000687047CB
:100C900000207047014BC058704700BF107AFF1FFB
:100CA000014B1868704700BF002004E070B52A4B64
:100CB0001C68C4F30B03240C63B140F2134293424B
:100CC00031D040F2194293422FD040F22142934258
:100CD0002DD10323214A0C2505FB03235D6893F9DD
:100CE000082042F201039C4224D0B4F5805F23D057
:100CF00041F201039C4221D041F203039C421FD0E8
:100D000041F207039C4208BF3122441E0C44013DBE
:100D10000B46A3421ED215F9016F581C96B103462B
:100D200000F8016CF5E70123D4E70223D2E73F2264
:100D30000B4DD6E73322E3E74122E1E75A22E4E70D
:100D40005922E2E72C2584421D7001D9981C5A7063
:100D5000401A70BD1846FBE7002004E0583A00082E
:100D60004C3A0008022802BF024B4FF080629A61A1
:100D7000704700BF00080240022802BF024B4FF438
:100D800080629A61704700BF00080240022801BFDC
:100D9000024A536983F4806353617047000802403C
:100DA00010B50023934203D0CC5CC4540133F9E75F
:100DB00010BD000030B5441E14F9010F0B4660B1A0
:100DC00093F90050854201F1010106D11AB993F956
:100DD0000020801A30BD013AEEE7002AF7D1104614
:100DE00030BD000002460346981A13F9011B002982
:100DF000FAD1704702440346934202D003F8011B24
:100E0000FAE77047024B1A78024B1A70704700BF1E
:100E10009829002000240020F8B5184C1848194DD6
:100E2000194E174F00F03AFC2146154800F062FCBD
:100E3000236816485A6DD2F8043843F00203C2F80A
:100E4000043801F0E3F82068114900F05FFD2368E1
:100E50005A6DD2F8043823F00203C2F804384FF474
:100E6000E1332B60002456F82400B84202D0294612
:100E700000F072FB0134042CF5D1F8BD703B000882
:100E80001437002084290020883A000840420F00CF
:100E9000C03B000838B50B4B1A780B4B53F8224077
:100EA0000A4B9C4205460CD0094B002118461422DF
:100EB000FFF7A0FF056001462046BDE8384000F07E
:100EC0004BBB38BD98290020883A00081437002011
:100ED00084290020026843681143016003B1184768
:100EE00070470000024AD36843F0C003D3607047E4
:100EF00000100140024AD36843F0C003D36070473A
:100F000000440040024AD36843F0C003D3607047F6
:100F1000005000402DE9F041D0F85C64F768336878
:100F2000DA0505469CB20DD5202383F311884FF4D2
:100F300000710430FFF7CEFF6FF48073336000233D
:100F400083F31188202383F3118805F1040814F03A
:100F50002F0333D183F31188380615D5210613D515
:100F6000202383F3118805F1380000F053FA00289C
:100F700046DA0821281DFFF7ADFF4FF67F733B408F
:100F8000F360002383F311887A060ED563060CD52F
:100F9000202383F31188EA6C2B6D9A4202D12B6CCB
:100FA000002B2FD1002383F31188D5F86424D36854
:100FB000002B31D01069BDE8F0411847230713D04A
:100FC00014F0080F0CBF00218021E00748BF41F05A
:100FD0002001A20748BF41F04001630748BF41F428
:100FE00080714046FFF776FFA406736805D595F833
:100FF00060142846194000F0BDFA3468A4B2A6E790
:101000007060BEE727F040073F041021281D3F0C09
:10101000FFF760FFF760C5E7BDE8F08108B503485A
:10102000FFF778FFBDE8084001F052BB9C29002083
:1010300008B50348FFF76EFFBDE8084001F048BB64
:10104000042E002008B50348FFF764FFBDE8084000
:1010500001F03EBB6C32002010B50E4C0E4A20460B
:10106000002100F057FA0D4BC4F85C340C4C0D4ACB
:101070002046002100F04EFA0B4BC4F85C340B4CB8
:101080000B4A0021204600F045FA0A4BC4F85C34B4
:1010900010BD00BF9C290020E50E00080010014093
:1010A000042E0020F50E0008004400406C320020A1
:1010B000050F00080050004038B5394D037C002969
:1010C00018BF0D46012B0446C0F8645410D1354BAF
:1010D000984242D1344B5A6C42F010025A645A6E14
:1010E00042F010025A665B6E0B21252000F06AF870
:1010F0002E4BD4F85C249A422B6802D02C498A42A9
:101100004BD12C4901EB5301B1FBF3F3A98808043F
:1011100042BF23F0070003F0070343EA4003936054
:10112000EB8843F040039BB213612B8943F001032A
:101130009BB2536141F4045343F02C03D36001F498
:10114000A05100231360B1F5806F136853680CBF82
:101150007F23FF2384F8603438BD174B98420CD1AD
:10116000114B1A6C42F400321A641A6E42F40032C7
:101170001A661B6E0B212620B8E7104B9842B7D198
:10118000094B1A6C42F480121A641A6E42F48012EF
:101190001A661B6E0B213520A8E70949B2E700BF8C
:1011A000B83A00089C290020003802400010014095
:1011B0000014014000BD0105042E00206C32002007
:1011C00080DE800200F1604300F01F02400903F559
:1011D000614309018000C9B200F1604083F8001347
:1011E00000F5614001239340C0F8803103607047EF
:1011F000F8B5154682680669AA420B46816938BF70
:101200008568761AB542044607D218462A46FFF783
:10121000C7FDA3692B44A3610DE011D932461846DE
:10122000FFF7BEFDAF1B3A46E1683044FFF7B8FD5B
:10123000E2683A44A261A3685B1BA3602846F8BD3C
:1012400018462A46FFF7ACFDE368E4E783682DE91A
:10125000F041044693421546266938BF85684069C7
:10126000361AB5420F4606D22A46FFF799FD636942
:101270002B4463610DE012D93246A5EB0608FFF757
:101280008FFD4246B919E068FFF78AFDE2684244E3
:101290006261A3685B1BA3602846BDE8F0812A4613
:1012A000FFF77EFDE368E4E710B50A440024C3615C
:1012B000029B006040608460C160816141610261A5
:1012C000036210BD08B582694369934201D1826807
:1012D00082B98268013282605A1C42611970426987
:1012E00003699A4201D3C3684361002100F0AAFE5A
:1012F000002008BD4FF0FF3008BD000070B520236E
:1013000004460E4683F31188A568A5B1A368A269B7
:10131000013BA360531CA36115782269934224BF4B
:10132000E368A361E3690BB120469847002383F388
:101330001188284670BD3146204600F073FE002813
:10134000E2DA85F3118870BD2DE9F74F05460F46A7
:1013500090469A46D0F81C90202686F311884FF0CC
:10136000000B144664B1224639462846FFF740FF79
:10137000034668B95146284600F054FE0028F1D0D3
:10138000002383F31188A8EB040003B0BDE8F08FBD
:10139000B9F1000F03D001902846C847019B8BF399
:1013A0001188E41A1F4486F31188DBE7C16081616C
:1013B0004161C3611144009B006040608260016133
:1013C00003627047F8B504460E461746202383F3A0
:1013D0001188A568A5B1A368013BA36063695A1C85
:1013E00062611E70236962699A4224BFE368636187
:1013F000E3690BB120469847002080F31188F8BDBF
:101400003946204600F00EFE0028E2DA85F3118806
:10141000F8BD0000836942699A4210B501D1826823
:101420007AB98268013282605A1C82611C78036931
:101430009A4201D3C3688361002100F003FE204675
:1014400010BD4FF0FF3010BD2DE9F74F05460F4698
:1014500090469A46D0F81C90202686F311884FF0CB
:10146000000B144664B1224639462846FFF7EEFECB
:10147000034668B95146284600F0D4FD0028F1D053
:10148000002383F31188A8EB040003B0BDE8F08FBC
:10149000B9F1000F03D001902846C847019B8BF398
:1014A0001188E41A1F4486F31188DBE70268436859
:1014B0001143016003B11847704700001430FFF773
:1014C00043BF00004FF0FF331430FFF73DBF000073
:1014D0003830FFF7B9BF00004FF0FF333830FFF767
:1014E000B3BF00001430FFF709BF00004FF0FF3119
:1014F0001430FFF703BF00003830FFF763BF000070
:101500004FF0FF323830FFF75DBF0000002070471A
:10151000FFF7A2BD37B50F4B036000234360836024
:10152000C360012304460374154600900B464FF434
:10153000007200F15C011430FFF7B6FE00942B46F8
:101540004FF4007204F5177104F13800FFF72EFF15
:1015500003B030BDCC3A000810B52023044683F315
:101560001188FFF7A9FD02232374002383F3118858
:1015700010BD000038B5C36904460D461BB90421EF
:101580000844FFF793FF294604F11400FFF79AFE81
:10159000002806DA201D4FF48061BDE83840FFF7CF
:1015A00085BF38BD026843681143016003B1184725
:1015B0007047000013B5446BD4F894341A6811785E
:1015C000042915D1217C022912D11979128901230C
:1015D0008B4013420CD101A904F14C0001F02EFE06
:1015E000D4F89444019B21790246206800F0DAF98E
:1015F00002B010BD143001F0B1BD00004FF0FF3358
:10160000143001F0ABBD00004C3001F083BE00008F
:101610004FF0FF334C3001F07DBE0000143001F07C
:101620007FBD00004FF0FF31143001F079BD0000A4
:101630004C3001F04FBE00004FF0FF324C3001F053
:1016400049BE0000D0F8942438B5136819780429ED
:10165000054601D0012038BD017C0229FAD112795A
:101660005C89012090400440F4D105F1140001F0A0
:1016700011FD02460028EDD0D5F894544FF4807344
:101680002868697900F07CF9204638BD406BFFF787
:10169000D9BF000000207047704700007FB5124B93
:1016A0000360002343608360C360012502260F4B63
:1016B000057404460290019300F1840229460096C5
:1016C0004FF48073143001F0C1FC094B0193029474
:1016D00000964FF4807304F52372294604F14C0000
:1016E00001F088FD04B070BDF43A00088D160008C2
:1016F000B51500080B68202282F311880A7903EBE4
:10170000820290614A79093243F822008A7912B143
:1017100003EB8203986102230374C0F8941400233E
:1017200083F311887047000038B5037F044613B176
:1017300090F85430ABB9201D01250221FFF732FF8C
:1017400004F1140025776FF0010100F087FC84F8A4
:10175000545004F14C006FF00101BDE8384000F036
:101760007DBC38BD10B5012104460430FFF71AFFD7
:101770000023237784F8543010BD000038B50446A8
:101780000025143001F07AFC04F14C00257701F0BB
:1017900049FD201D84F854500121FFF703FF204626
:1017A000BDE83840FFF74EBF90F8443003F06003C7
:1017B000202B19D190F84520212A0AD0222A4FF057
:1017C00000030ED0202A0FD1084A82630722C26389
:1017D00004E0064B83630723C363002303640120F3
:1017E00070478363C363F9E700207047012400203A
:1017F000D0F8943437B51A681178042904461AD100
:10180000017C022917D11979128901238B401342D7
:1018100011D100F14C05284601F0C4FD58B101A9D1
:10182000284601F00BFDD4F89444019B217902462F
:10183000206800F0B7F803B030BD000000EB810372
:10184000F7B59C6905460E46F4B1202383F3118851
:1018500005EB8607201D0821FFF7A4FEFB685B69E6
:101860001B684C3413B1204601F0F6FC01A9204658
:1018700001F0E4FC024648B1019B3146284600F0E5
:1018800091F8002383F3118803B0F0BDFB685A6917
:101890001268002AF5D01B8A013B1340F1D105F1F3
:1018A0004402EAE7093138B550F82140DCB1202381
:1018B00083F31188D4F894241368527903EB8203DC
:1018C000DB689B695D6845B104216018FFF76AFE1B
:1018D000294604F1140001F0E7FB2046FFF7B2FEB1
:1018E000002383F3118838BD7047000000F0A8BFC3
:1018F0000123037000234360C36183620362C362F8
:1019000043620363038143817047000038B5044696
:10191000202383F3118800254160C560056145617E
:10192000856100F09DFF0223237085F3118838BD87
:1019300070B500EB810305465069DA600E46144627
:1019400018B110220021FFF755FAA06918B1102232
:101950000021FFF74FFA31462846BDE8704001F0FC
:1019600049B80000028902F001020281428902F0B6
:1019700001024281002202614261826101F0CEB81F
:10198000F0B400EB81044789E4680125A4698D4027
:101990003D43458123600023A2606360F0BC01F0F9
:1019A000E9B80000F0B400EB81040789E468012580
:1019B00064698D403D43058123600023A26063601C
:1019C000F0BC01F063B9000070B5022300250446A5
:1019D0000370A0F84C5080F84E5080F84F500581AD
:1019E0004581C56005614561856180F8345000F02E
:1019F0009DFF63681B6823B129462046BDE87040FF
:101A0000184770BD436802781B6880F85020052293
:101A100002700BB10421184770470000436890F82A
:101A200050201B6802700BB1052118477047000059
:101A300090F8343070B5044613B1002380F8343088
:101A400004F14402204601F08BF863689B6863BB95
:101A500094F8445015F0600615D194F8453005F01F
:101A60007F0545EA032540F202339D4200F00E81D6
:101A70005BD8022D00F0DC803FD8002D00F087807D
:101A8000012D00F0CF800021204601F0C1FA002195
:101A9000204601F0B3FA63681B6813B106212046A3
:101AA0009847062384F8343070BD204698470028B4
:101AB000CED094F84B2094F84A3043EA0223E26BEC
:101AC000934238BFE36394F94430E56B002B4FF049
:101AD000200380F2FD80002D00F0EC80092284F8C4
:101AE000342083F311880021E36BA26B2046FFF7BB
:101AF00059FF002383F3118870BDB5F5817F00F095
:101B0000B180B5F5407F49D0B5F5807FBBD194F861
:101B10004630012BB7D1B4F84C3023F00203A4F8BF
:101B20004C30A663E6632664C3E740F201639D423E
:101B30001ED8B5F5C06F3BD2B5F5A06FA3D1B4F8F0
:101B40004430B3F5A06F0ED194F8463084F84E308F
:101B5000204600F043FF63681B6813B10121204653
:101B60009847032323700023A363E3632364A0E760
:101B7000B5F5106F32D040F602439D4252D0B5F514
:101B8000006F80D104F14F03A363012324E004F12B
:101B90004C03A3630223E36325648AE794F8463089
:101BA000012B7FF470AFB4F84C3043F00203B6E77A
:101BB00094F84920616894F848304D6894F84710CB
:101BC00043EA0223204694F84620A84700283FF421
:101BD0005AAF4368A3630368E363A4E72378042B45
:101BE00010D1202383F311882046FFF7BBFE86F334
:101BF0001188636884F84F601B68032121700BB162
:101C00002046984794F84630002BACD084F84F30EB
:101C10000423237063681B68002BA4D00221204694
:101C20009847A0E7374BA3630223E36300239DE7B4
:101C300094F8481011F0800F204601F00F010ED0EB
:101C400000F080FF012806D002287FF41CAF2E4B45
:101C5000A363E06367E72D4BA363E56363E700F0ED
:101C600063FFEFE794F84630002B7FF40CAF94F855
:101C7000483013F00F013FF476AF1A06204602D524
:101C800001F0DAF96FE701F0CDF96CE794F846302E
:101C9000002B7FF4F8AE94F8483013F00F013FF4B6
:101CA00062AF1B06204602D501F0B2F95BE701F0F6
:101CB000A5F958E7142284F8342083F311882B46C1
:101CC0002A4629462046FFF75BFE85F3118870BD42
:101CD0005DB1152284F8342083F311880021E36B71
:101CE000A26B2046FFF74CFE03E70B2284F834205A
:101CF00083F311882B462A4629462046FFF752FED9
:101D0000E3E700BF243B00081C3B0008203B000821
:101D100038B590F834300446152B29D8DFE803F0A5
:101D20003E28282828283E28280B29392828282812
:101D3000282828283E3E90F84B1090F84A20C36B84
:101D400042EA01229A4214D9C268128AB3FBF2F520
:101D500002FB15356DB9202383F311882B462A46E3
:101D60002946FFF71FFE85F311880A2384F83430D3
:101D700038BD142384F83430202383F311880023E2
:101D80001A4619462046FFF7FBFD002383F311880E
:101D900038BD036C03B198470023E7E7002101F049
:101DA00037F90021204601F029F963681B6813B157
:101DB0000621204698470623D8E7000090F83420F3
:101DC000152A38B5044622D80123934040F64162D3
:101DD00013421DD113F480150FD19B0217D50B238D
:101DE00080F83430202383F311882B462A46294675
:101DF000FFF7D8FD85F3118838BDC3689B695B6820
:101E00002BB9036C03B19847002384F8343038BDF4
:101E1000002101F0FDF80021204601F0EFF8636891
:101E20001B6813B10621204698470623EDE7000002
:101E3000024B00221B605B609A607047D436002022
:101E4000002303748268054B1B6899689142FBD29A
:101E50005A6803604260106058607047D4360020B2
:101E600008B5202383F31188037C032B05D0042BB2
:101E70000DD02BB983F3118808BD436900221A6085
:101E80004FF0FF334361FFF7DBFF0023F2E790E8F9
:101E90000C001A6002685360F2E70000002303742C
:101EA0008268054B1B6899689142FBD85A680360A9
:101EB0004260106058607047D4360020054B1969A5
:101EC0000874186802681A6053601861012303746B
:101ED000FEF71ABAD436002030B54B1C87B0054641
:101EE0000A4C10D023690A4A01A800F0D3F828460A
:101EF000FFF7E4FF049B13B101A800F007F9236981
:101F0000586907B030BDFFF7D9FFF8E7D436002095
:101F1000611E000838B50C4D41612B6981689A68D3
:101F20009142044603D8BDE83840FFF789BF184600
:101F3000FFF786FF01232C61014623742046BDE88C
:101F40003840FEF7E1B900BFD4360020044B1A68D0
:101F50001B6990689B68984294BF002001207047DD
:101F6000D436002010B5084C236820691A68226016
:101F70005460012223611A74FFF790FF0146206923
:101F8000BDE81040FEF7C0B9D436002082600222BE
:101F900002740022427470478368A3F17C0243F804
:101FA0000C2C026943F83C2C426943F8382C074A50
:101FB00043F81C2CC26843F8102C022203F8082CAA
:101FC000002203F8072CA3F1180070472103000832
:101FD00010B5202383F31188FFF7DEFF00210446AC
:101FE000FFF798FF002383F31188204610BD0000FF
:101FF000024B1B6958610F20FFF760BFD4360020E9
:10200000202383F31188FFF7F3BF000008B50146D2
:10201000202383F311880820FFF75EFF002383F35A
:10202000118808BD49B1064B42681B6918605A60A7
:10203000136043600420FFF74FBF4FF0FF3070473D
:10204000D43600200368984206D01A6802605060B7
:1020500059611846FFF7F4BE7047000038B50446D2
:102060000D462068844200D138BD036823605C605F
:102070004561FFF7E5FEF4E7054B03F114025A61F1
:102080009A614FF0FF32DA6100221A62704700BF96
:10209000D4360020F8B503614FF08043C2605C6A1B
:1020A000194B1A46022952F8145F38BF0221954293
:1020B00006461F460AD1586198611C62056045605A
:1020C00081600819BDE8F84001F08EB9186AAB6864
:1020D000241A0C1902D3E41A2D6804E09C4202D29F
:1020E000204401F08FF9AB689C42F4D86B687360B0
:1020F00035601E606E60B460A9684FF0FF33091B45
:10210000A960FB61F8BD00BFD436002010B41B4CA1
:10211000234653F8141F814210D0416802680A60B8
:10212000026851609A424FF00001C16003D0936889
:1021300081680B4493605DF8044B70470A686261E4
:1021400000209A425360C86003D15DF8044B01F04F
:1021500053B993688868034493604FF08042206AC3
:10216000526A121A9342E6D9991A012998BF931C10
:1021700018445DF8044B01F045B900BFD436002087
:1021800000207047FEE70000704700004FF0FF306E
:1021900070470000022906D0032906D0012906480D
:1021A00018BF0020704705487047032A9ABF0448AB
:1021B00000EBC200002070471C3C0008D03B000828
:1021C0000824002070B5044608460D46FEF70AFEB6
:1021D000C6B22046013403780BB9184670BD3246AA
:1021E0002946FEF7E7FD0028F3D1012070BD00006D
:1021F0002DE9F04F81469BB008460C461646FEF787
:10220000F1FD3C49C5B22046FFF7DCFF08B10535BA
:10221000EDB239492046FFF7D5FF08B11035EDB2D0
:10222000632D01AF0CD8DFF8DCA0DFF8DCB03D4651
:1022300094F80080B8F1000F1CD185F8008003E00D
:102240002146384601F0F6FB3846FEF7CBFDC0B21A
:10225000431C5B0089E8480033700323737000233C
:1022600002361946DAB2904206F102063AD81BB09D
:10227000BDE8F08FB8F1250F2FD107221D49204668
:10228000FEF798FD58B9DBF800202A60DBF804203F
:102290006A60DBF80820AA6007340C35C8E708221A
:1022A00015492046FEF786FDB8B91448AA1C10F857
:1022B000011F134B4FEA111E01F00F011EF80AE037
:1022C00011F80A1002F802EC984202F8011C02F11F
:1022D0000202ECD118350834AAE785F800800134F1
:1022E0000135A5E7FA5C06F8022C06F8011C01335B
:1022F000B8E700BF783B0008803B00080F7AFF1F5B
:102300001B7AFF1F963B0008893B000808B5202375
:1023100083F311880348FFF76BFA002383F31188D6
:1023200008BD00BF1437002010B50446052916D893
:10233000DFE801F016150316161D202383F311881C
:102340000E4A0121FFF7F4FA20460D4A0221FFF759
:10235000EFFA0C48FFF712FA002383F3118810BD3F
:10236000202383F311880748FFF7DEF9F4E72023E1
:1023700083F311880348FFF7F5F9EDE7283B0008E0
:102380004C3B00081437002038B50C4D0C4C0D495F
:102390002A4604F10800FFF72BFF05F1CA0204F1F9
:1023A00010000949FFF724FF05F5CA7204F118006F
:1023B0000649BDE83840FFF71BBF00BFDC3B0020EB
:1023C00008240020A83B0008B23B0008803B00081E
:1023D000BFF34F8F024AD368DB03FCD4704700BFC2
:1023E000003C024008B5094B1B7873B9FFF7F0FFBA
:1023F000074B1A69002ABFBF064A5A6002F18832A9
:102400005A601A6822F480621A6008BD3A3E0020C1
:10241000003C02402301674508B50B4B1B7893B97C
:10242000FFF7D6FF094B1A6942F000421A611A6899
:1024300042F480521A601A6822F480521A601A68B4
:1024400042F480621A6008BD3A3E0020003C02401F
:102450000B2870B513D80B4A0B4C137863B90B4E8D
:102460004FF0006144F8231056F8235001330C2B31
:102470002944F7D10123137054F8200070BD0020C7
:1024800070BD00BF6C3E00203C3E00203C3C00087C
:10249000014B53F8200070473C3C00080C2070476B
:1024A0000B2810B5044601D9002010BDFFF7D0FF5E
:1024B000064B53F824301844C21A0BB9012010BD42
:1024C00012680132F0D1043BF6E700BF3C3C000843
:1024D0000B2810B504461ED8FFF77AFFFFF782FFDE
:1024E0000E49F323CB60FFF773FFC300DBB243F465
:1024F000007343F002030B610B6943F480330B61FB
:10250000FFF766FFFFF7A4FFFFF786FF2046BDE851
:102510001040FFF7C5BF002010BD00BF003C0240C7
:102520002DE9F84312F00103154643D10244B2F1FC
:10253000016F3FD22C4B1B6813F001033AD02B4C98
:10254000FFF750FFF323E360FFF742FF40F201275C
:10255000032D16D8254C0F46401A40F20118EB1BEC
:102560000B44012B00EB0706236926D823F0010357
:102570002361FFF751FF0120BDE8F883043D0430DB
:10258000E6E78307E6D1236923F4407323612369D7
:102590003B43236151F8046B0660BFF34F8FFFF795
:1025A00017FF03689E42E9D0236923F001032361EA
:1025B000FFF732FF0020BDE8F88323F44073236166
:1025C000236943EA08032361B94637F8023B3380A5
:1025D000BFF34F8FFFF7FCFE3688B9F80030B6B274
:1025E000B342BCD0E0E700BF00380240003C0240EC
:1025F000084908B50B7828B153B9FFF7F3FE01235A
:102600000B7008BD23B1BDE808400870FFF704BF98
:1026100008BD00BF3A3E0020014B53F82000704730
:10262000502800400A4B1A6F120407D41A6F42F464
:1026300000721A671A6F42F400421A67054A13685B
:1026400043F48073136000B2034B43F820107047CB
:10265000003802400070004050280040014B1868CC
:10266000704700BF5028004001460020FFF7DABF46
:1026700038B5094B1B689B000CD5084B084D01224F
:102680001A700024E0B2FFF7C7FF45F824000134B8
:10269000082CF7D138BD00BF74380240903E0020AE
:1026A000703E0020014B1878704700BF903E00201C
:1026B000064A536823F001035360EFF3098368333C
:1026C00083F30988002383F31188704730EF00E01B
:1026D00010B5202383F31188104B5B6813F400635B
:1026E00018D0F1EE103AEFF309844FF0807344F8FC
:1026F0004C3C0B4BDB6844F8083CA4F1680383F3C3
:102700000988FFF723FC18B1064B44F8503C10BD74
:10271000054BFAE783F3118810BD00BF00ED00E020
:1027200030EF00E031030008340300087047000078
:10273000FEE70000084A094B09498B4204D3094AC5
:102740000021934205D3704752F8040F43F8040B5D
:10275000F3E743F8041BF4E7E43D00088841002058
:102760008841002088410020836D30B500229D689B
:10277000446D11464FF0FF3004EB42130132954295
:10278000C3F80019C3F81019C3F80809C3F8001BEF
:10279000C3F8101BC3F8080BEED24FF00113C4F8B6
:1027A0001C3830BD890141F02001016103699B069D
:1027B000FCD4122000F0AEBE204B03EB80022DE9CA
:1027C000F047D2F80CE05D6DDEF81420461CD2F81C
:1027D00000C005EB063605EB4018516861450BD388
:1027E000D5F83428012303FA00F022EA0000C5F8E6
:1027F00034081846BDE8F087BEF81040ACEB010382
:10280000A34228BF2346D8F81849A4B2B3EB840FDB
:1028100010D894681F46A4F1040959F804AFC6F80B
:1028200000A0042F01D9043FF7E71C440B44946037
:102830005360D2E70020BDE8F08700BF943E00203F
:1028400010B5054C2046FFF753F84FF0A0436365E1
:10285000024BA36510BD00BF943E0020903C0008D1
:102860000378012B70B5054650D12A4B446D984230
:102870001BD1294B5A6B42F080025A635A6D42F0C9
:1028800080025A655A6D5A6942F080025A615A694B
:1028900022F080025A610E2143205B69FEF792FC10
:1028A0001E4BE3601E4BC4F800380023C4F8003E02
:1028B000C02323606E6D4FF40413A3633369002BB0
:1028C000FCDA012333610C2000F024FE3369DB07BE
:1028D000FCD4122000F01EFE3369002BFCDA002627
:1028E000A6602846FFF740FF6B68C4F81068DB68F5
:1028F000C4F81468C4F81C684BB90A4BA3614FF0C4
:10290000FF336361A36843F00103A36070BD064B0E
:10291000F4E700BF943E002000380240401400401D
:1029200003002002003C30C0083C30C0F8B5446DC4
:10293000054600212046FFF735FFA96D00234FF023
:1029400001128F68C4F834384FF00066C4F81C28B0
:102950004FF0FF3004EB431201339F42C2F800698D
:10296000C2F8006BC2F80809C2F8080BF2D20B6873
:102970006A6DEB65636210231361166916F0100629
:10298000FBD1122000F0C6FDD4F8003823F4FE631A
:10299000C4F80038A36943F4402343F01003A36153
:1029A0000923C4F81038C4F814380A4BEB604FF010
:1029B000C043C4F8103B084BC4F8003BC4F810698E
:1029C000C4F80039EB6D03F1100243F48013EA659B
:1029D000A362F8BD6C3C000840800010426D90F886
:1029E0004E10D2F8003823F4FE6343EA0113C2F814
:1029F000003870472DE9F0410EB200EB86080D4615
:102A0000D8F80C100F6807F00303022B50D0032BEB
:102A100050D03D4A3D4F012B18BF1746446D4FEA39
:102A2000451E04EB0E030022C3F8102B8A6905F142
:102A3000100C002A40D04A8A05F158035B013A4342
:102A4000E2500123D4F81C2803FA0CF31343A644E4
:102A50004A69C4F81C380023CEF8103905F13F0349
:102A6000002A39D00A8A898B9208012988BF4A43F3
:102A7000C16D04EB8303561841EA0242C66529463C
:102A80005A602046FFF78EFED8F80C301B8A43EAC6
:102A900085531F4305F148035B01E7500123D4F838
:102AA0001C2803FA05F51543C4F81C58BDE8F0814D
:102AB000174FB3E7174FB1E704EB4613D3F8002BDA
:102AC00022F40042C3F8002BD4F81C28012303FA97
:102AD0000CF322EA0303BAE704EB83030E4A5A60BD
:102AE00004EB461629462046FFF75CFED6F800396F
:102AF00023F40043C6F80039D4F81C38012202FA46
:102B000005F523EA0505CFE70080001000800410DA
:102B10000080081000800C1000040002826D126812
:102B2000C265FFF721BE00005831436D49015B5873
:102B300013F4004004D013F4001F14BF012002203E
:102B4000704700004831436D49015B5813F4004061
:102B500004D013F4001F14BF0120022070470000AE
:102B600000EB8101CB68196A0B6813604B685360F6
:102B70007047000000EB810330B5DD68AA69136877
:102B8000D36019B9402B84BF402313606B8A14684B
:102B9000426D1C44013CB4FBF3F46343033323F064
:102BA000030302EB411043EAC44343F0C043C0F8BF
:102BB000103B2B6803F00303012B09B20ED1D2F8AE
:102BC000083802EB411013F4807FD0F8003B14BFAB
:102BD00043F0805343F00053C0F8003B02EB411236
:102BE000D2F8003B43F00443C2F8003B30BD000084
:102BF0002DE9F041244D6E6D06EB40130446D3F8E9
:102C0000087BC3F8087B38070AD5D6F814381907AB
:102C100006D505EB84032146DB6828465B689847A8
:102C2000FA072FD5D6F81438DB072BD505EB84032C
:102C3000D968CCB98B69488A5E68B6FBF0F200FBB4
:102C400012628AB91868DA6890420DD2121A83E8C3
:102C50001400202383F311880B482146FFF78AFFD5
:102C600084F31188BDE8F081012303FA04F26B8933
:102C700023EA02036B81CB6823B121460248BDE8F9
:102C8000F0411847BDE8F081943E002000EB81033D
:102C900070B5DD68436D6C692668E6604A0156BB15
:102CA0001A444FF40020C2F810092A6802F0030207
:102CB000012A0AB20ED1D3F8080803EB421410F42B
:102CC000807FD4F8000914BF40F0805040F00050DD
:102CD000C4F8000903EB4212D2F8000940F00440A6
:102CE000C2F80009D3F83408012202FA01F10143C5
:102CF000C3F8341870BD19B9402E84BF402020603D
:102D000020682E8A841940F00050013C1A44B4FB1C
:102D1000F6F440EAC440C6E7F8B504461E48456DDF
:102D200005EB4413D3F80869C3F80869F10717D510
:102D3000D5F81038DA0713D500EB8403D9684B694E
:102D40001F68DA68974218D2D21B00271A605F60AA
:102D5000202383F311882146FFF798FF87F311881A
:102D6000330617D5D5F834280123A340134211D0D8
:102D70002046BDE8F840FFF71FBD012303FA04F227
:102D8000038923EA020303818B68002BE8D02146E4
:102D90009847E5E7F8BD00BF943E002096482DE92E
:102DA000F84F456D6E69AB691E4016F4805F6E6129
:102DB000044605D0FEF708FEBDE8F84FFFF788BCD3
:102DC000002E12DAD5F8003E8B489B071EBFD5F8BF
:102DD000003E23F00303C5F8003ED5F8043823F085
:102DE0000103C5F80438FEF719FE370502D58248FD
:102DF000FEF708FEB0040CD5D5F8083813F0060F1E
:102E0000EB6823F470530CBF43F4105343F4A05306
:102E1000EB60310704D56368DB680BB176489847EF
:102E2000F2025AD4B3020CD5D4F85480DFF8C8A10A
:102E300000274FF00109A36D9B68F9B28B4280F027
:102E40008780F70619D5616D0A6AC2F30A1702F086
:102E50000F0302F4F012B2F5802F00F0A180B2F55A
:102E6000402F0AD104EB830301F58051DB68186A17
:102E700000231A469F4240F087803003D5F8184857
:102E800013D5E10302D50020FFF7B2FEA20302D55D
:102E90000120FFF7ADFE630302D50220FFF7A8FE75
:102EA000270302D50320FFF7A3FE750384D5E007AF
:102EB00002D50020FFF730FFA10702D50120FFF760
:102EC0002BFF620702D50220FFF726FF23077FF5BD
:102ED00073AF0320FFF720FF6EE7D4F85480DFF8CC
:102EE00018A100274FF00109A36D9B685FFA87FBCB
:102EF0005B4597D308EB4B13D3F8002902F440222B
:102F0000B2F5802F22D1D3F80029002A1EDAD3F897
:102F1000002942F09042C3F80029D3F80029002A82
:102F2000FBDB5946606DFFF73DFC228909FA0BF384
:102F300022EA0303238104EB8B03DB689B6813B154
:102F40005946504698475846FFF736FC0137CBE7BD
:102F500008EB4112D2F8003B03F44023B3F5802F75
:102F600010D1D2F8003B002B0CDA628909FA01F388
:102F700022EA0303638104EB8103DB68DB680BB1A6
:102F800050469847013756E79C0708BF0A68072B49
:102F900098BF027003F101039CBF120A013069E778
:102FA000023304EB830201F5805152689069026894
:102FB000D0F808C04068A2EB000E002210469742ED
:102FC0000AD104EB830463689B699A683A449A6067
:102FD0005A6817445F6050E712F0030F08BF086893
:102FE000964588BF8CF8000002F1010284BF000AF8
:102FF0000CF1010CE3E700BF943E0020436D03EBAE
:103000004111D1F8003B43F40013C1F8003B704775
:10301000436D03EB4111D1F8003943F40013C1F8BB
:1030200000397047436D03EB4111D1F8003B23F4A5
:103030000013C1F8003B7047436D03EB4111D1F819
:10304000003923F40013C1F80039704730B5039CF0
:103050000172043304FB0325C361049B0363002155
:10306000059B00604060C16042610261856104624D
:1030700042628162C162436330BD00000022416A46
:1030800041610161C2608262C2626FF00101FEF7BC
:10309000E5BF000003694269934203D1C2680AB1E7
:1030A00000207047181D704703691960C26801321B
:1030B000C260C269134482690361934224BF436AB8
:1030C00003610021FEF7BEBF38B504460D46E36834
:1030D0003BB16269131D1268A3621344E3620020CE
:1030E00038BD237A33B929462046FEF79BFF0028D6
:1030F000EDDA38BD6FF00100FBE70000C368C2697C
:10310000013BC3604369134482694361934224BF16
:10311000436A436100238362036B03B1184770471E
:1031200070B52023044683F31188866A3EB9FFF701
:10313000CBFF054618B186F31188284670BDA36AF7
:10314000E26A13F8015BA362934202D32046FFF7C1
:10315000D5FF002383F31188EFE700002DE9F84F36
:1031600004460E4690469946202787F3118800258D
:10317000AA46D4F828B0BBF1000F09D14946204631
:10318000FFF7A2FF20B18BF311882846BDE8F88F26
:10319000A16AE36AA8EB050B5B1A9B4528BF9B4617
:1031A000BBF1400F1BD9334601F1400251F8040B2B
:1031B00043F8040B9142F9D1A36A40334036A3622D
:1031C0004035A26AE36A9A4202D32046FFF796FF8F
:1031D0008AF311884545D8D287F31188C9E730466C
:1031E0005A46FDF7DDFDA36A5B445E44A3625D447D
:1031F000E7E7000010B5029C0172043303FB0421D1
:10320000C36100238362C362039B0363049B00606A
:103210004060C46042610261816104624262436352
:1032200010BD0000026AC260426A4261026100226F
:103230008262C2626FF00101FEF710BF436902694A
:103240009A4203D1C2680AB100207047184650F86C
:10325000043B0B6070470000C368C2690133C36060
:103260004369134482694361934224BF436A4361C3
:103270000021FEF7E7BE000038B504460D46E368BE
:103280003BB123691A1DA262E2691344E362002084
:1032900038BD237A33B929462046FEF7C3FE0028FD
:1032A000EDDA38BD6FF00100FBE70000036919603B
:1032B000C268013AC260C2691344826903619342E1
:1032C00024BF436A036100238362036B03B1184781
:1032D0007047000070B5202304460E4683F3118822
:1032E000856A35B91146FFF7C7FF10B185F311881C
:1032F00070BDA36A1E70A36AE26A01339342A3629F
:1033000004D3E16920460439FFF7D0FF002080F3A1
:10331000118870BD2DE9F84F04460D4691469A4636
:103320004FF0200888F311880026B346A76A4FB9EA
:1033300051462046FFF7A0FF20B187F311883046A1
:10334000BDE8F88FA06AE76AA9EB06033F1A9F421F
:1033500028BF1F46402F1BD905F1400355F8042B09
:1033600040F8042B9D42F9D1A36A4033A362403652
:10337000A26AE36A9A4204D3E16920460439FFF75E
:1033800095FF8BF311884E45D9D288F31188CDE78C
:1033900029463A46FDF704FDA36A3B443D44A36237
:1033A0003E44E5E7026943699A4203D1C3681BB909
:1033B000184670470023FBE7836A002BF8D0043BD4
:1033C0009B1AF5D01360C368013BC360C3691A44FC
:1033D000836902619A4224BF436A036100238362C6
:1033E0000123E5E700F02EB94FF080430022586337
:1033F0001A610222DA6070474FF080430022DA60DF
:10340000704700004FF0804358637047FEE70000AC
:1034100010B5174CFEF70CFDFEF72EFE8022154965
:103420002046FEF7B3FD012344F8180C0374124B39
:10343000124AD96821F4E0610904090C0A431049D1
:10344000DA60CA6842F08072CA600E490A6842F0C7
:1034500001020A601022DA77202283F8222000235A
:1034600083F3118862B60848BDE81040FEF7B0BD8E
:10347000FC3600209C3C000800ED00E00003FA054B
:10348000F0ED00E0001000E0A43C00082DE9F84F4A
:103490001F4C4FF00008656904F11407C1464FF056
:1034A0008043266A5B6AAA689E1B96421DD34FF032
:1034B000200AAA68236AD5F80CB0134423622B684B
:1034C000BB425F60A6EB02066361C5F80C8001D1C8
:1034D000FFF792FF89F311882869D8478AF311888A
:1034E0006569AB689E42E4D2D9E76269BA420CD002
:1034F000916823628E1B9660A86802282CBF18185A
:10350000981CBDE8F84FFFF77DBFBDE8F88F00BFFE
:10351000D4360020034B59685A68521A9042FBD89F
:10352000704700BF001000E04B6843608B68836009
:10353000CB68C3600B6943614B6903628B6943626B
:103540000B6803607047000008B5224B22481A69D7
:1035500040F2FF110A431A611A6922F4FF7222F045
:1035600001021A611A691A6B0A431A631A6D0A4337
:103570001A651A4A1B6D1146FFF7D6FF184802F16B
:103580001C01FFF7D1FF174802F13801FFF7CCFF0C
:10359000154802F15401FFF7C7FF144802F170010A
:1035A000FFF7C2FF124802F18C01FFF7BDFF11487F
:1035B00002F1A801FFF7B8FF0F4802F1C401FFF7BD
:1035C000B3FF0E4802F1E001FFF7AEFFBDE808408F
:1035D00000F0A2B80038024000000240C43C0008DD
:1035E0000004024000080240000C024000100240AB
:1035F0000014024000180240001C0240002002405B
:1036000008B500F0F9F9FFF703FFFFF731F8BDE85F
:103610000840FEF7B9BE0000704700004FF080433D
:1036200010B51A69920708D500241C61202383F382
:103630001188FFF72BFF84F31188BDE81040FFF7D6
:1036400047B80000104B1A6C42F001021A641A6E5F
:1036500042F001021A660D4A1B6E936843F00103A3
:1036600093604FF0804353229A624FF0FF32DA6248
:1036700000229A615A63DA605A6001225A61082175
:103680001A601C20FDF79EBD00380240002004E0B7
:103690001F4B1A696FEAC2526FEAD2521A611A6955
:1036A000C2F308021A614FF0FF301A695A69586173
:1036B00000215A6959615A691A6A62F080521A6285
:1036C0001A6A02F080521A621A6A5A6A58625A6A70
:1036D00059625A6A1A6C42F080521A641A6E42F0A9
:1036E00080521A661A6E0B4A106840F4807010609F
:1036F000186F00F44070B0F5007F1EBF4FF48030AB
:1037000018671967536823F40073536000F054B9C5
:103710000038024000700040304B4FF080521A6475
:103720002F4A4FF4404111601A6842F001021A60BA
:103730001A689207FCD59A6822F003029A60274B18
:1037400019469A6812F00C02FBD1186800F0F900D3
:1037500018609A601A6842F480321A600B689B0302
:10376000FCD54B6F43F001034B671C4B5A6F90071E
:10377000FCD51C4A5A601A6842F080721A60184AD6
:1037800053685904FCD5154B1A689201FCD5164AAA
:103790009A60164B1A68164B9A42164B1BD1164A62
:1037A0001168164A914216D140F205121A600B4B6D
:1037B0009A6842F002029A609A6802F00C02082AA3
:1037C000FAD15A6C42F480425A645A6E42F48042F2
:1037D0005A665B6E704740F20572E7E700380240B8
:1037E000007000400854400700948838002004E02E
:1037F00011640020003C024000ED00E041C20F4196
:10380000084A08B5536911680B4003F0010353617E
:1038100023B1054A13680BB150689847BDE80840CA
:10382000FEF756BF003C014008410020084A08B599
:10383000536911680B4003F00203536123B1054A39
:1038400093680BB1D0689847BDE80840FEF740BFC9
:10385000003C014008410020084A08B5536911683E
:103860000B4003F00403536123B1054A13690BB104
:1038700050699847BDE80840FEF72ABF003C014068
:1038800008410020084A08B5536911680B4003F04D
:103890000803536123B1054A93690BB1D069984776
:1038A000BDE80840FEF714BF003C0140084100207D
:1038B000084A08B5536911680B4003F010035361BF
:1038C00023B1054A136A0BB1506A9847BDE8084016
:1038D000FEF7FEBE003C014008410020174B10B52A
:1038E0005C691A68144004F478725A61A30604D51E
:1038F000134A936A0BB1D06A9847600604D5104A00
:10390000136B0BB1506B9847210604D50C4A936B8F
:103910000BB1D06B9847E20504D5094A136C0BB183
:10392000506C9847A30504D5054A936C0BB1D06C35
:103930009847BDE81040FEF7CBBE00BF003C0140F9
:10394000084100201A4B10B55C691A68144004F451
:103950007C425A61620504D5164A136D0BB1506D55
:103960009847230504D5134A936D0BB1D06D984742
:10397000E00404D50F4A136E0BB1506E9847A104B2
:1039800004D50C4A936E0BB1D06E9847620404D5EF
:10399000084A136F0BB1506F9847230404D5054AAA
:1039A000936F0BB1D06F9847BDE81040FEF790BE03
:1039B000003C014008410020062108B50846FDF7FB
:1039C00001FC06210720FDF7FDFB06210820FDF77D
:1039D000F9FB06210920FDF7F5FB06210A20FDF77A
:1039E000F1FB06211720FDF7EDFB06212820BDE89D
:1039F0000840FDF7E7BB000008B5FFF749FE00F0FF
:103A00000DF8FDF785FDFDF771FFFDF745FEFFF7AA
:103A100003FEBDE80840FFF7E5BC000000230449B1
:103A20001A465A50C8180833802B4260F9D17047A3
:103A300008410020034611F8012B03F8012B002A4E
:103A4000F9D17047121012131211000053544D3364
:103A500032463F3F3F000000000000004C3A0008A3
:103A60003F00000013040000983A00083F000000E7
:103A700019040000A23A00083F00000021040000E1
:103A8000AC3A00083F000000143700209C290020B9
:103A9000042E00206C32002053544D333246343013
:103AA000780053544D3332463432780053544D33FA
:103AB00032463434365858000096000000000000AA
:103AC00000000000000000000000000000000000F6
:103AD000D9140008C514000801150008ED140008E9
:103AE000F9140008E5140008D1140008BD140008FA
:103AF0000D1500080000000011160008FD15000853
:103B00003916000825160008311600081D16000891
:103B100009160008F51500089516000800000000B9
:103B20000100000000000000020000000000000092
:103B30003D180008A518000840004000AC3B0020DC
:103B4000BC3B002002000000000000000300000059
:103B500000000000E918000800000000100000004C
:103B6000CC3B00200000000001000000000000002D
:103B7000943E00200101020025424F41524425009D
:103B80002553455249414C25004633354C696768F9
:103B9000746E696E670030313233343536373839F8
:103BA00041424344454600004172647550696C6F60
:103BB000740025424F415244252D424C0000000024
:103BC0002923000895210008A91700080D230008E3
:103BD00043000000D83B000809024300020100C076
:103BE0003209040000010202010005240010010551
:103BF00024010001042402020524060001070582B5
:103C0000030800FF09040100020A00000007050183
:103C10000240000007058102400000001200000081
:103C2000243C0008120110010200004083044057A8
:103C30000002010203010000040309040040000027
:103C400000400000004000000040000000000100B3
:103C5000000002000000020000000200000002005C
:103C6000000002000000020000000200000000004E
:103C7000311A0008111D0008BD1D00084000400059
:103C8000F43E0020F43E002001000000043F00202C
:103C90008000000040010000030000006D61696EBB
:103CA00000000000BC3C0008103F0020084100203C
:103CB000010000000D3400080000000069646C651C
:103CC00000000000A000A80200000000AAAAAAAA02
:103CD00050001400FFFF00000077000070A70A00EA
:103CE0000000000000000000AAAAAAAA000000002C
:103CF000FFFF0000000000000000000000001002B4
:103D000000000000AAAAAAAA00000001FFFB000010
:103D1000000000000000080020000000000000007B
:103D2000AAAAAAAA10000000FFFF000000080000D5
:103D3000000000000000000000000000AAAAAAAADB
:103D400000000000FFFF0000000000000000000075
:103D50000000000000000000AAAAAAAA00000000BB
:103D6000FFFF000000000000000000000000000055
:103D700000000000AAAAAAAA00000000FFFF00009D
:103D80000000000000000000000000000000000033
:103D90000A00000000000000030000000000000016
:103DA0000000000000000000000000000000000013
:103DB0000000000000000000000000000000000003
:103DC000FF0096000000000804000000383C0008D6
:103DD00000000000000000000000000000000000E3
:083DE0000000000000000000DB
:00000001FF
